:100000000C94CE020C9412030C9412030C94120361
:100010000C9412030C9412030C9412030C9412030C
:100020000C9412030C9412030C94B60D0C94880ECD
:100030000C9412030C9412030C9412030C941203EC
:100040000C9412030C9492220C9412030C9412033D
:100050000C9412030C94251C0C9412030C941203A0
:100060000C9412030C9412030C9412030C941203BC
:100070000C9412030C9412030C9412030C941203AC
:100080000C9412030C9412030C9412030C9412039C
:100090000C9412030C9412030C9412030C9412038C
:1000A0000C9412030C9412030C941203F50E170F08
:1000B0000510170F05105C0F7F0F0510D40FE70F09
:1000C000B612B612E512E5121B133B136C146C1436
:1000D00046136C14F613F6135D146C146C1466144A
:1000E0000314031403140314031403140314031458
:1000F0000314031403140314031403140314031448
:1001000015142214291430143A140000F0A12E0002
:100110002B002900E100354100001E0014000400FE
:100120001D713400E2001F001A0016001B00E104DC
:100130004C00200008000700060050002A002100A3
:100140001500090019004F004D00220017000A0099
:10015000050000006574E30001540000007F00000A
:100160004A004F000354000000770000E200230023
:100170001C000B00110000002971240018000D0064
:10018000100052004B0025000C000E0036005100FC
:100190002C00260012000F0037002F002800270037
:1001A00013003342387130004E002D00310034000E
:1001B000E500C10000000100010001000100010094
:1001C00000003A001E0220022202010001003B0052
:1001D0001F0221022302010001003C002F0226021F
:1001E0002F00010001003D00300227023000010015
:1001F00001003E003102350035020000010001001F
:1002000001000000010000000100010001000000E9
:100210000100000001003F005200510024020000D4
:1002200001004000240021001E00010001004100E7
:10023000250022001F003700010042002600230095
:10024000200027000100430025022E0231002E006D
:100250000100440045000100010001000000010010
:100260000100010001000100000001000100010087
:1002700001000100010001000100F2000100010085
:10028000F5000100F000F1000100F400F4000100AD
:100290000100F3000100F500010001000100010070
:1002A0000100000001000100010000000100000049
:1002B0000100010001000000010000000100010038
:1002C0000100F20001000000010001000100F10046
:1002D0000100A900010001000100F000AC00AA002B
:1002E000B70001000100F300AB00A800B600010058
:1002F0000100010001000100010001000100AE0049
:1003000001000100000000000000000000000000EB
:10031000000000001E0014000400000000000000A7
:100320001F001A001600000019000000200008003D
:100330000700000006000000210015000900000071
:1003400000000000220017000A000000C4000000A6
:10035000000000000000000000000100000000009C
:10036000000000000100000023001C000B00000042
:1003700001000000240018000D0001000100000031
:1003800025000C000E0001001000000026001200E5
:100390000F000000110000002700130033000000D0
:1003A0000000010001002F003400000000001603CF
:1003B0004500720067006F0044006F007800200065
:1003C00045005A00000016034500720067006F00E8
:1003D00044006F007800200045005A00000004032C
:1003E000090409026D00040100A0FA0904000001DB
:1003F00003010100092111010001223F00070581CD
:100400000308000A09040100010301020009211187
:10041000010001224D000705820308000A090402B9
:10042000000103000000092111010001223600072C
:1004300005830308000A0904030001030000000902
:100440002111010001223900070584031000011267
:1004500001100100000008EDFE0713010001020079
:100460000105010906A101050719E029E715002585
:100470000195087501810205081901290595057581
:10048000019102950175039101050719002977155E
:10049000002501957875018102C005010980A1013F
:1004A000850216010026B7001A01002AB700751050
:1004B00095018100C0050C0901A101850316010009
:1004C000269C021A01002A9C02751095018100C029
:1004D00005010902A1010901A10005091901290568
:1004E00015002501950575018102950175038101AE
:1004F0000501093009311581257F950275088106AE
:1005000009381581257F950175088106050C0A3883
:10051000021581257F950175088106C0C005010976
:1005200006A101050719E029E715002501950875C1
:1005300001810295017508810105081901290595B8
:1005400005750191029501750391010507190029AF
:10055000FF150025FF950675088100C0000000000A
:1005600000000000000000010204060A0F17202C02
:100570003A4A5D71879DB3C7DAE9F5FCFFFCF5E9FE
:10058000DAC7B39D87715D4A3A2C20170F0A06041B
:1005900002010000000000000000000011241FBE46
:1005A000CFEFDAE0DEBFCDBF04B603FE24C08091FA
:1005B000FB019091FC01A091FD01B091FE018730FB
:1005C000904BA740B04BB9F41092FB011092FC0184
:1005D0001092FD011092FE0114BE84B7877F84BF84
:1005E00088E10FB6F89480936000109260000FBE0F
:1005F000E0E0FFE3099511E0A0E0B1E0E2EBF8E410
:1006000002C005900D92A433B107D9F711E0A4E31D
:10061000B1E001C01D92AB3FB107E1F70E94FA0AB9
:100620000C9457240C9400001092B9008AE0809337
:10063000B800089594EA9093BC009091BC0097FF95
:10064000FCCF9091B900987F983021F0903111F053
:1006500081E008958093BB0084E88093BC00809182
:10066000BC0087FFFCCF8091B900887F883111F0F2
:10067000803471F780E0089584E98093BC00809114
:10068000BC0084FDFCCF08958093BB0084E8809378
:10069000BC008091BC0087FFFCCF9091B900987F8F
:1006A00081E0983209F480E0089584E88093BC00EA
:1006B0008091BC0087FFFCCF8091BB0008958091A2
:1006C0000101811115C080E40E941A038093010189
:1006D00081110CC082E10E944403809301018111C9
:1006E00005C08FEF0E944403809301010E943C03E8
:1006F00084B1807F84B985B1807F85B98AB1837FD9
:100700008AB98BB1837F8BB93E98469808950E9431
:100710001A05809301010E945F0380B38C7080BB37
:1007200081B3836F81BBA5E3B1E0E3E4F1E08EE048
:100730008E0F11921D928E13FCCF0C940405BF9264
:10074000CF92DF92EF92FF920F931F93CF93DF939D
:1007500080910101882379F0809134018F5F80932B
:100760003401811108C00E941A0580930101811192
:1007700002C00E94AC0405E311E0C0E0D0E0DD243B
:10078000D39482E0C82EEE24E394F12CC730D10537
:1007900000F580910101811164C080E40E941A0378
:1007A00080930101811112C082E10E944403809371
:1007B000010181110BC0C7010C2E01C0880F0A94E2
:1007C000EAF780950E944403809301010E943C0354
:1007D00048C0CA30A1F028F4C83059F0C93061F0DF
:1007E00005C0CC3089F070F0CD3089F0209A28987F
:1007F00010C0219A29980DC0229A2A980AC0239ADB
:100800002B9807C0529A01C0539A5B9802C03E9A37
:10081000469890EA9A95F1F79FB1799902C082E0E3
:1008200001C080E091709D25982B7C9902C084E0E6
:1008300001C080E0892B7D9902C038E001C030E022
:10084000832B7E9902C020E101C020E0822B9FB162
:100850009095991F9927991F9295990F907E892BB2
:100860000FC080910101811149C080E40E941A03E8
:1008700080930101882379F1B12C0E943C038B2DD8
:10088000F8019081981719F08083C09200010E94AE
:100890005F0321960F5F1F4FCE30D10509F076CF51
:1008A00080910001882361F18150809300018823A9
:1008B00039F08FE99FE00197F1F700C0000020C0F8
:1008C000A3E4B1E0E5E3F1E0CF01825F91919D9374
:1008D0008E13FCCF15C083E10E9444038093010175
:1008E0008111CACF81E40E941A0380930101811112
:1008F000C3CF0E945503B82EB094BFCF80E0C0CFC5
:100900000E94AA0481E0DF91CF911F910F91FF9087
:10091000EF90DF90CF90BF900895E82FF0E0ED5B6F
:10092000FE4F8081089508950F931F93CF93DF9317
:10093000C3E4D1E010E00C2F025F899190E00E94A7
:100940004B1B180F0C13F9CF812FDF91CF911F9103
:100950000F9108950C947A0556985E9825982D98D5
:1009600026982E9827982F988FEF90E090938900E3
:100970008093880090938B0080938A0090938D00E1
:1009800080938C00259A2D9A2FEF80E792E02150DA
:1009900080409040E1F700C00000269A2E9A2FEF89
:1009A00080E792E0215080409040E1F700C00000D5
:1009B000279A2F9A2FEF80E792E0215080409040B5
:1009C000E1F700C0000025982D982FEF80E792E016
:1009D000215080409040E1F700C0000026982E98FA
:1009E0002FEF80E792E0215080409040E1F700C077
:1009F000000027982F9856985E9825982D9826984D
:100A00002E9827982F98089589EA8093800089E08E
:100A10008093810024982C983F988AB18F748AB96A
:100A20006E98479A8BB1806B8BB9769A0E94AC0412
:100A30000C94790580E2809301018091510181112C
:100A40000EC00E94140381E0809351012FEF83EDCB
:100A500090E3215080409040E1F700C0000080E426
:100A60000E941A038093010181112EC00E94440349
:100A700080930101811128C00E94440380930101E9
:100A8000811122C08FE30E944403809301018111F0
:100A90001BC00E943C0380E40E941A038093010162
:100AA000811112C08CE00E944403809301018111E6
:100AB0000BC00E94440380930101811105C08FE3A4
:100AC0000E944403809301010E943C038091010134
:100AD000089561110BC0FC018281882321F085EE0D
:100AE0000E945A1103C085EE0E94221280E090E01D
:100AF000089508956091BD017091BE018091BF017C
:100B00009091C0010E94571B56985E9825982D9889
:100B100026982E9827982F98813019F0823021F04E
:100B20000895259A2D9A0895269A2E9A089581E07F
:100B3000089581E008950C94990508950F931F93EB
:100B4000CF93DF938C01FC01C081D181CE010E9443
:100B5000D019BE010E944706EC01B8010E949B0516
:100B6000882309F48DC0F8018281882309F44AC0E2
:100B700080915D0181111FC0C431F0E5DF0709F0EC
:100B800051C00E949D0581E080935D010E94EF1B92
:100B900090935C0180935B01109254011092560176
:100BA00010925501109258011092570110925A015B
:100BB0001092590165C080915B0190915C010E9487
:100BC000FB1B883C910570F480915401E82FF0E004
:100BD000EE0FFF1FEB5AFE4FD183C0838F5F8093D0
:100BE00054014EC0C43880E5D80721F0C538D0453F
:100BF00001F13AC0F8018281882341F0109252013C
:100C000082E01EC0C438E0E5DE0759F5809152014C
:100C1000811106C086E20E945A1186E20E942212C9
:100C200082E01CC0C438F0E5DF0741F3C538D04589
:100C3000D9F4F8018281882331F01092530180E2C7
:100C40000E9471121DC080915301811106C087E27C
:100C50000E945A1187E20E94221280E20E947812BA
:100C60000FC0C538D04529F381E0809352018093AD
:100C70005301C801DF91CF911F910F910C949705FB
:100C800080E0DF91CF911F910F910895089596E034
:100C9000799FF001112494E5899FE00DF11D112445
:100CA000E60FF11DEE0FFF1FE25FFE4F859194915D
:100CB0000895880F991FFC01E657F04085919491A3
:100CC0000895880F991FFC01E65FFE4F859194916E
:100CD00008950F931F93CF93DF93EC01811520E3C9
:100CE000920750F5C11580E2D80708F0C3C0CB3B8E
:100CF000D10590F4C83AD10508F06AC0C53AD105CB
:100D000008F05BC0C430D10508F0D0C1219709F0CC
:100D1000CAC101E010E00AC2CF3FD10511F008F0CE
:100D2000C5C1C03FD10508F0A2C0CE01805E9109C7
:100D3000089708F4BBC1B7C1C13090E5D90709F4E1
:100D4000A2C020F5C0318FE4D80770F4C11590E43B
:100D5000D90708F094C0C11521E3D20708F0A3C158
:100D6000DD278E01106CE2C1C115D04509F09BC191
:100D70000E94D7148FEF94E32CE0815090402040E4
:100D8000E1F700C000000E944A1CD0C1C11597E5E0
:100D9000D90758F4C03121E5D20708F01CC1C4318D
:100DA00080E5D80708F475C07EC1CE019057811543
:100DB000904108F078C1DF7073C1C53AD10509F4DC
:100DC00077C1C63AD10509F076C102E810E4AEC198
:100DD000C83AD10509F472C1C93AD10509F471C103
:100DE000CA3AD10509F470C1CB3AD10509F46FC1F3
:100DF000CC3AD10509F46EC1CD3AD10509F46DC1E3
:100E0000C03BD10509F46CC1CE3AD10509F46BC1E0
:100E1000CF3AD10509F46AC1C13BD10509F469C1D2
:100E2000C23BD10509F468C1C33BD10509F467C1D0
:100E3000C43BD10509F466C1C53BD10509F465C1C0
:100E4000C63BD10509F464C1C73BD10509F463C1B0
:100E5000C83BD10509F462C1C93BD10509F461C1A0
:100E6000CA3BD10509F460C100E014E45FC18E0102
:100E700010655CC1CE019F700E94610658C1DF7091
:100E80008E01106A53C18091DA0181608093DA018A
:100E90004DC10E94EF1D811102C00E94D51D0E940C
:100EA0000C1E90E09093FB018093FA01C23080E524
:100EB000D80721F48091FA01816086C0C43090E5A2
:100EC000D90721F48091FA0182607EC0C63020E506
:100ED000D20721F48091FA01846076C0C83080E5A1
:100EE000D80719F48091FA0127C0CA3090E5D907D4
:100EF00021F48091FA01806167C0CC3020E5D207EF
:100F000021F48091FA0180625FC0CE3080E5D8077D
:100F100021F48091FA01806457C0C03190E5D9076F
:100F200021F48091FA0180684FC0C23120E5D207D8
:100F300029F48091FA018460886046C0C33080E55E
:100F4000D80721F48091FA018E7F3EC0C53090E52C
:100F5000D90721F48091FA018D7F36C0C73020E592
:100F6000D20721F48091FA018B7F2EC0C93080E531
:100F7000D80719F48091FA0126C0CB3090E5D90743
:100F800021F48091FA018F7E1FC0CD3020E5D20779
:100F900021F48091FA018F7D17C0CF3080E5D8070A
:100FA00021F48091FA018F7B0FC0C13190E5D90700
:100FB00021F48091FA018F7707C0C331D04531F415
:100FC0008091FA018B7F877F8093FA018091FA01EB
:100FD0000E94101EABC08D2F99278F7099278130EA
:100FE0009105D9F49E012370332702C0880F991F01
:100FF0002A95E2F79C688E0144E0000F111F4A9584
:10100000E1F700271370802B912B53E0CC0FDD1FED
:101010005A95E1F7C076DD272FC08230910531F473
:10102000DC2FCC278E01016F106A80C083309105C0
:1010300069F4CE018370992701E010E002C0000F2F
:10104000111F8A95E2F7C8019C680FC08430910592
:10105000B9F4CE018370992701E010E002C0000FBF
:10106000111F8A95E2F7C8019A6823E0CC0FDD1FB3
:101070002A95E1F7C07ED7708C010C2B1D2B56C032
:101080008530910531F4DC2FCC278E01046F106A76
:101090004DC0069709F04AC0CF71DD27DC2FCC2761
:1010A0008E01106243C000E010E040C08E013EC0DF
:1010B00001E810E43BC003E810E438C002EE14E499
:1010C00035C009EE14E432C00AEE14E42FC005EB7B
:1010D00014E42CC006EB14E429C007EB14E426C08A
:1010E0000CEC14E423C00DEC14E420C003E815E478
:1010F0001DC00AE815E41AC002E915E417C004E9A6
:1011000015E414C001E216E411C003E216E40EC0B7
:1011100004E216E40BC005E216E408C006E216E499
:1011200005C007E216E402C00AE216E4C801DF9136
:10113000CF911F910F91089596E0799FF0011124AE
:1011400094E5899FE00DF11D1124E60FF11DEE0FCE
:10115000FF1FE25FFE4F85919491803E9105E0F480
:10116000803C910558F58133910509F46FC048F42E
:101170008932910509F463C08A32910509F46DC082
:1011800072C089339105E9F082389105D1F0853339
:10119000910509F44DC067C0833E910581F138F493
:1011A000803E9105B9F0823E9105D9F05CC0863E43
:1011B000910561F1873E9105A1F155C00E94590644
:1011C00008952091FA0120FD02C021FF4CC080EE5D
:1011D00090E049C08091FA0180FFF9CF89E390E067
:1011E00042C08091FA0182FF0EC08091FA0184FF13
:1011F00003C080E090E037C083EE90E034C080917F
:10120000FA0182FFF2CF82EE90E02DC08091FA01C8
:1012100083FF0BC08091FA0184FDEBCF87EE90E055
:1012200022C08091FA0183FFF5CF86EE90E01BC0CB
:101230008091FA0185FF07C089E290E014C0809197
:10124000FA0185FFF9CF85E390E00DC08091FA01A6
:1012500086FF07C08AE290E006C08091FA0186FF0F
:10126000F9CF81E390E00E946906089508950C94F7
:10127000360980916E010895CF93DF9300D01F92BD
:10128000CDB7DEB79C018091F101843019F593E070
:1012900099833B832A839093E9008FEF9091E80034
:1012A000815095FD06C095ED9A95F1F700008111EA
:1012B000F5CF8091E80085FF0DC040E050E063E08D
:1012C00070E0CE0101960E94A60B8091E8008E7717
:1012D0008093E8000F900F900F90DF91CF910895C9
:1012E000CF93DF9300D01F92CDB7DEB72091F101ED
:1012F000243021F522E029839B838A8383E0809335
:10130000E9008FEF9091E800815095FD06C095EDC2
:101310009A95F1F700008111F5CF8091E80085FFE3
:101320000DC040E050E063E070E0CE0101960E9405
:10133000A60B8091E8008E778093E8000F900F90C5
:101340000F90DF91CF9108952091F1012430F1F4B5
:1013500022E02093E9002FEF3091E800215035FD85
:1013600006C035ED3A95F1F700002111F5CF209137
:10137000E80025FF0BC040E050E065E070E00E940F
:10138000A60B8091E8008E778093E8000895CF93B4
:10139000DF93EC019091F101943009F046C0809107
:1013A0000C018823D9F080910D018823B9F0909326
:1013B000E9008FEF9091E800815095FD06C095E11E
:1013C0009A95F1F700008111F5CF8091E80085FF33
:1013D0002CC040E050E060E170E017C081E08093F5
:1013E000E9008FEF9091E800815095FD06C095EDE2
:1013F0009A95F1F700008111F5CF8091E80085FF03
:1014000014C040E050E068E070E0CE010E94A60BFE
:101410008091E8008E778093E80080E1FE01AEE5E0
:10142000B1E001900D928A95E1F7DF91CF91089597
:101430008091F001811109C00E943B0D0E94980D1E
:101440008091E20084608093E20008951092F001A0
:10145000089508950C947F220E94E01B0E9485222B
:101460000E943E100C94370942E061EC81E00E943A
:10147000B50C42E061EC82E00E94B50C42E061EC08
:1014800083E00E94B50C42E161EC84E00C94B50C61
:101490008091F301833009F455C030F4813071F04C
:1014A000823009F48EC008958A3009F47AC08B30F6
:1014B00009F460C0893009F09CC020C08091F2011D
:1014C000813A09F096C08091E800877F8093E80018
:1014D0008091F6019091F701892B21F460E18EE56E
:1014E00091E003C060E080E090E070E00E94F10BCA
:1014F0008091E8008B778093E80008958091F20155
:10150000813209F076C08091F6019091F701009741
:1015100019F0039709F06DC08091E800877F8093F0
:10152000E8008091E80082FD05C08091F101811101
:10153000F8CF5FC08091F10080936E018091E80048
:101540008B7753C08091F201813A09F052C08091AB
:10155000F6019091F701892B09F04BC08091E800CA
:10156000877F8093E8008091E80080FFFCCF809126
:101570000C0136C08091F2018132D9F58091F601DB
:101580009091F701892BA9F58091E800877F8093DE
:10159000E8000E94EA0C8091F40180930C010C9405
:1015A000D7148091F201813221F58091E800877F84
:1015B0008093E8000E94EA0C8091F50180936F010E
:1015C00008958091F201813AA1F48091E800877F2B
:1015D0008093E8008091E80080FFFCCF80916F014C
:1015E0008093F1008091E8008E778093E8000C945E
:1015F000EA0C089584B7877F84BF88E10FB6F8941A
:1016000080936000109260000FBE90E080E80FB6FB
:10161000F89480936100909361000FBE0E948D103A
:101620000E943B0D0E94980D8091E200846080939F
:10163000E20078940E941E100E948F1082E091E0D8
:101640000E9439100E946D228091F101853069F469
:101650000E94A71B8091EF018823B1F30E94D21B47
:10166000882391F30E94900BEFCF0E949510ECCF4E
:10167000292F332723303105C9F064F42130310597
:1016800081F02230310509F043C08DE690E022EE72
:1016900033E042C021323105F1F02232310541F10F
:1016A00037C082E190E02FE434E036C099278130E2
:1016B000910541F08230910541F0892B49F5EEED1D
:1016C000F3E005C0E6ECF3E002C0EEEAF3E084915B
:1016D00090E09F0121C06430D8F4E62FF0E0EE0FD7
:1016E000FF1FEE5DFE4F2081318189E090E014C044
:1016F000643070F470E0FB01EE0FFF1FE65EFE4FFA
:1017000020813181FB01EA5EFE4F808190E004C0C0
:1017100080E090E020E030E0FA01318320830895FA
:1017200080E189BD82E189BD09B400FEFDCF8091D1
:10173000D8008F7D8093D8008091E00082608093F4
:10174000E0008091E00081FDFCCF0895CF92DF9210
:10175000EF92FF920F931F93CF93DF93EC018B01D6
:101760006A010E94090D811133C0C114D10439F0FE
:10177000F60180819181081B190BC80FD91FE12C3C
:10178000F12C0115110519F18091E80085FD16C0B5
:101790008091E8008E778093E800C114D10449F06D
:1017A000F60180819181E80EF91EF182E08285E0E8
:1017B0000FC00E94090D882321F30AC089918093EC
:1017C000F10001501109FFEFEF1AFF0ADACF80E0B4
:1017D000DF91CF911F910F91FF90EF90DF90CF900D
:1017E00008952091F8013091F9012617370748F044
:1017F0006115710539F42091E8002E772093E800F7
:1018000001C0B90140E061157105A9F12091F10114
:10181000222309F443C0253009F442C02091E80096
:1018200023FD40C02091E80022FD32C02091E80055
:1018300020FFE9CF4091F3002091F20030E0342BFB
:10184000FC01CF016115710559F02830310540F4D4
:1018500081918093F100615071092F5F3F4FF1CF6B
:1018600041E02830310509F040E02091E8002E7772
:101870002093E800C8CF4111C9CF0AC08091F1017F
:10188000882361F0853061F08091E80083FD0AC013
:101890008091E80082FFF2CF80E0089582E0089511
:1018A00083E0089581E008952091F8013091F901D5
:1018B0002617370748F06115710539F42091E800C3
:1018C0002E772093E80001C0B901FC0120E06115EA
:1018D000710591F18091F101882309F440C08530B0
:1018E00009F43FC08091E80083FD3DC08091E8008D
:1018F00082FD2FC08091E80080FFE9CF2091F300A6
:101900008091F20090E0922B6115710559F08830BA
:10191000910540F424912093F100319661507109B2
:101920000196F2CF21E0089709F020E08091E800CD
:101930008E778093E800CBCF2111CCCF0AC0809165
:10194000F101882361F0853061F08091E80083FD2A
:101950000AC08091E80082FFF2CF80E0089582E023
:10196000089583E0089581E00895982F973058F501
:101970009093E900981739F07091EC002091ED00F8
:101980005091F00003C0242F762F50E021FF19C0A2
:101990003091EB003E7F3093EB003091ED003D7FC6
:1019A0003093ED003091EB0031603093EB00709399
:1019B000EC002093ED005093F0002091EE0027FF03
:1019C00007C09F5FD3CF8F708093E90081E00895B7
:1019D00080E008958091F20187FF11C08091E800B6
:1019E00082FD05C08091F1018111F8CF11C0809175
:1019F000E8008B770BC08091F101882349F080913A
:101A0000E80080FFF8CF8091E8008E778093E800AF
:101A100008952091E4003091E50095E64091EC00B6
:101A2000842F817040FF22C08091E80080FD1CC09F
:101A30008091F101882391F0853091F08091EB0045
:101A400085FD10C04091E4005091E5004217530716
:101A500029F39A01915011F784E0089582E00895E6
:101A600083E0089581E0089580E008954091E800C2
:101A700042FFDECF08950E94A90D0E94B10DE0EE55
:101A8000F0E0808181608083E8EDF0E080818F77F5
:101A9000808319BCA7EDB0E08C918E7F8C93808100
:101AA0008F7E80831092F00108950F931F93CF9340
:101AB000DF930E94A90D0E94B10DC8EDD0E088818E
:101AC0008F77888388818068888388818F7D8883E9
:101AD00019BC1092F1011092ED011092EF011092D9
:101AE000EE0100EE10E0F80180818B7F8083888119
:101AF0008160888342E060E080E00E94B50CE1EE06
:101B0000F0E080818E7F8083E2EEF0E08081816072
:101B10008083808188608083F80180818E7F8083CC
:101B2000888180618883DF91CF911F910F91089503
:101B3000E8EDF0E080818F7E8083E7EDF0E080814A
:101B40008160808384E082BF81E08093F0010C9407
:101B5000550DE8EDF0E080818E7F80831092E200E9
:101B600008951092DA001092E10008951F920F92EA
:101B70000FB60F9211242F933F934F935F936F9360
:101B80007F938F939F93AF93BF93EF93FF93809136
:101B9000E10082FF0BC08091E20082FF07C08091CC
:101BA000E1008B7F8093E1000E941D108091DA009C
:101BB00080FF1FC08091D80080FF1BC08091DA0099
:101BC0008E7F8093DA008091D90080FF0DC080E184
:101BD00089BD82E189BD09B400FEFDCF81E080931B
:101BE000F1010E94180A05C019BC1092F1010E946F
:101BF000260A8091E10080FF19C08091E20080FFF9
:101C000015C08091E2008E7F8093E2008091E20017
:101C100080618093E2008091D80080628093D80038
:101C200019BC85E08093F1010E942A0A8091E100AD
:101C300084FF30C08091E20084FF2CC080E189BD28
:101C400082E189BD09B400FEFDCF8091D8008F7D6F
:101C50008093D8008091E1008F7E8093E100809195
:101C6000E2008F7E8093E2008091E20081608093A9
:101C7000E2008091ED01882311F084E007C080919B
:101C8000E30087FD02C081E001C083E08093F101A1
:101C90000E942C0A8091E10083FF29C08091E2001C
:101CA00083FF25C08091E100877F8093E10082E07F
:101CB0008093F1011092ED018091E1008E7F80937D
:101CC000E1008091E2008E7F8093E2008091E2004B
:101CD00080618093E20042E060E080E00E94B50C09
:101CE0008091F00088608093F0000E94290AFF91A3
:101CF000EF91BF91AF919F918F917F916F915F9184
:101D00004F913F912F910F900FBE0F901F901895FC
:101D10001F920F920FB60F9211242F933F934F9360
:101D20005F936F937F938F939F93AF93BF93CF9363
:101D3000DF93EF93FF93C091E900CF708091EC00A7
:101D4000D82FD17080FDD0E81092E9008091F0008A
:101D5000877F8093F00078940E94CC0E1092E90067
:101D60008091F00088608093F000CD2BCF70C093FD
:101D7000E900FF91EF91DF91CF91BF91AF919F91DA
:101D80008F917F916F915F914F913F912F910F9024
:101D90000FBE0F901F9018951F93CF93DF93CDB771
:101DA000DEB7AA970FB6F894DEBF0FBECDBFE2EF45
:101DB000F1E088E08E0F9091F10091938E13FBCFAC
:101DC0000E94480A8091E80083FF1FC18091F201C0
:101DD0009091F301492F50E04A30510508F015C1A8
:101DE000FA01EA5AFF4F0C940724803881F08238B8
:101DF00009F00BC18091F6018F708093E90080910A
:101E0000EB0085FB882780F91092E90006C08091DD
:101E1000EE019091EF01911182609091E800977F1F
:101E20009093E8008093F1001092F100C8C0282F31
:101E30002D7F09F0EAC0882319F0823061F0E5C0F7
:101E40008091F401813009F0E0C0933009F080E026
:101E50008093EF012BC08091F401811127C0809104
:101E6000F6018F7009F4D1C08093E9002091EB0056
:101E700020FF1CC0933021F48091EB00806214C0DD
:101E80009091EB0090619093EB0021E030E0A9018C
:101E900002C0440F551F8A95E2F74093EA00109262
:101EA000EA008091EB0088608093EB001092E900DB
:101EB0008091E800877F86C08111A7C01091F4014E
:101EC0001F778091E3008078812B8093E3008091DD
:101ED000E800877F8093E8000E94EA0C8091E80088
:101EE00080FFFCCF8091E30080688093E3001111B4
:101EF00002C082E001C083E08093F10186C0805877
:101F0000823008F082C08091F4019091F5018C3DFF
:101F100053E0950779F583E08A838AE289834FB796
:101F2000F894DE01139620E03EE051E2E32FF0E06A
:101F300050935700E49120FF03C0E295EF703F5F9C
:101F4000EF708E2F90E0EA3010F0C79601C0C09677
:101F50008D939D932F5F243149F74FBF8091E80007
:101F6000877F8093E8006AE270E0CE0101960E94CC
:101F7000F10B14C0AE014F5F5F4F6091F6010E94FC
:101F8000380BBC01009709F440C09091E800977F9E
:101F90009093E80089819A810E94540C8091E80016
:101FA0008B778093E80031C0803879F58091E80024
:101FB000877F8093E8008091ED018093F10080910C
:101FC000E8008E778093E8000E94EA0C1EC0811121
:101FD0001CC09091F4019230C0F48091E800877F9A
:101FE0008093E8009093ED010E94EA0C8091ED014E
:101FF000811106C08091E30087FD02C081E001C02D
:1020000084E08093F1010E94340A8091E80083FF0C
:102010000AC08091E800877F8093E8008091EB0000
:1020200080628093EB00AA960FB6F894DEBF0FBED5
:10203000CDBFDF91CF911F9108950895CF938091E7
:10204000F1018823A1F0C091E900CF709091EC00DC
:10205000892F817090FD80E8C82B1092E900809153
:10206000E80083FD0E94CC0ECF70C093E900CF91B1
:10207000089590937501809374010895E09174011F
:10208000F0917501309721F00190F081E02D0994D5
:1020900080E00895E0917401F0917501309721F08E
:1020A0000280F381E02D09940895E0917401F0918C
:1020B0007501309721F00480F581E02D0994089591
:1020C00020917201309173018217930771F0909300
:1020D000730180937201E0917401F0917501309762
:1020E00021F00680F781E02D099408952091700178
:1020F000309171018217930771F090937101809371
:102100007001E0917401F0917501309721F0008425
:10211000F185E02D0994089508950C948C100E9487
:10212000E61B0E9487030C94A81C9F92AF92BF925B
:10213000CF92DF92EF92FF920F931F93CF93DF9393
:1021400000D000D000D0CDB7DEB70E949F030DE0D5
:1021500010E0AA24A394B12C902E802F0E948D040D
:10216000980129583E4F6901F901F080F826A1F441
:102170000150110988F78FEF89838A831B820E949F
:10218000EF1B8160782F9D838C8349815A816B81FD
:102190008D810E942C112FC09091DA0191FF04C013
:1021A0008E830E9493048E8125E030E0A501022EEB
:1021B00001C0440F0A94EAF7E42E4F21C1F02983AD
:1021C0009A828E2191E009F490E09B830E94EF1B9C
:1021D0008160782F9D838C8349815A816B818D81A9
:1021E0000E942C11F6018081E826E08204C0215073
:1021F0003109E0F6BDCF0E948F1F109176010E9439
:102200003E101817B9F00E943E1080937601269672
:102210000FB6F894DEBF0FBECDBFDF91CF911F91F7
:102220000F91FF90EF90DF90CF90BF90AF909F9075
:102230000C94370926960FB6F894DEBF0FBECDBFBB
:10224000DF91CF911F910F91FF90EF90DF90CF9092
:10225000BF90AF909F900895CF93DF93CDB7DEB737
:102260002B970FB6F894DEBF0FBECDBF4F835887B4
:1022700069877A878B87DE01119686E0FD011192CE
:102280008A95E9F785E0FE01379601900D928A95CF
:10229000E1F749815A816B817C818D819E810E9409
:1022A00075172B960FB6F894DEBF0FBECDBFDF912A
:1022B000CF910895CF93882309F4C2C0C82F8238E4
:1022C00059F40E943E1081FDBBC089E30E944F1A61
:1022D0000E941C1B89E30CC0833879F40E943E10D5
:1022E00080FDAEC083E50E944F1A0E941C1B83E54F
:1022F0000E94911ACF910C941C1B843859F40E94AF
:102300003E1082FD9DC087E40E944F1A0E941C1B54
:1023100087E4EECF8CEF8C0F813A48F48C2F0E942B
:10232000D22181118DC08C2F0E944F1AE3CF80E201
:102330008C0F883048F4C77081E001C0880FCA95BF
:10234000EAF70E94D51AD6CF8BE58C0F833078F44C
:10235000C53A29F0C63A31F083E890E005C081E83B
:1023600090E002C082E890E0CF910C94601088E584
:102370008C0F833108F064C0C83A39F1C93A41F191
:10238000CA3A49F1CB3A51F1CC3A59F1CD3A61F11F
:10239000C03B69F1CE3A71F1CF3A79F1C13B81F19D
:1023A000C23B89F1C33B91F1C43B99F1C53BA1F11B
:1023B000C63BA9F1C73BB1F1C83BB9F1C93BC1F17B
:1023C000CA3BC9F180E090E038C082EE90E035C0B1
:1023D00089EE90E032C08AEE90E02FC085EB90E06D
:1023E0002CC086EB90E029C087EB90E026C08CECF7
:1023F00090E023C08DEC90E020C083E891E01DC008
:102400008AE891E01AC082E991E017C084E991E07E
:1024100014C081E292E011C083E292E00EC084E237
:1024200092E00BC085E292E008C086E292E005C02F
:1024300087E292E002C08AE292E0CF910C9476109B
:10244000CF910895882309F44BC0823859F40E9433
:102450003E1081FF45C089E30E944F1A0E941C1B59
:1024600089E30CC0833871F40E943E1080FF38C0AD
:1024700083E50E944F1A0E941C1B83E50E94911A5B
:102480000C941C1B843859F40E943E1082FF28C013
:1024900087E40E944F1A0E941C1B87E4EFCF9CEF39
:1024A000980F913A58F390E2980F983050F4877053
:1024B00091E001C0990F8A95EAF7892F0E94DB1AF3
:1024C000DFCF9BE5980F933020F480E090E00C94F0
:1024D0006010885A833120F480E090E00C947610EC
:1024E0000895882321F00E94D51A0C941C1B08958E
:1024F000882321F00E94DB1A0C941C1B08957F9204
:102500008F929F92AF92BF92CF92DF92EF92FF9203
:102510000F931F93CF93DF931F92CDB7DEB77C014C
:10252000C62E772EFC01058102950F7012811111C4
:102530000E94F21A0E94481A882379F0112369F048
:1025400080E28C0D883048F082E00E94311A0E94AF
:10255000481A91E0D82ED92601C0D12CE72DE2955A
:10256000EF70F0E0E05AFF4F0C940724872D807F36
:10257000072D0F70882311F00295007F112389F039
:10258000002309F490C180E28C0D883020F4802F64
:102590000E94D51A03C0802F0E94E51A0E941C1BBE
:1025A00082C18C2D0E942212002309F495C180E281
:1025B0008C0D883020F4802F0E94DB1A03C0802FFE
:1025C0000E94EB1A0E941C1B87C1972D907F872DBC
:1025D0008F70903211F08295807FCC2021F0F1E055
:1025E000CF16B1F01EC0112349F0002309F414C125
:1025F000013009F011C10E94051B6EC1002319F0C2
:10260000013009F469C189830E94081B89810AC1CC
:10261000112321F0023008F05FC1FEC001115CC13E
:1026200001C1112321F0002309F4F6C03CC10023AD
:1026300009F4F8C03EC1872D86958695837090E099
:10264000009719F0019761F047C1112321F08C2DFB
:10265000972D937002C080E090E00E9460103CC112
:10266000112321F08C2D972D937002C080E090E013
:102670000E94761031C18C2D112319F00E94971EF3
:1026800002C00E94FF1E0E94841F26C1872D8370F6
:1026900009F052C0111120C18C2D8295869587704A
:1026A000880F880F9C2D9F70892E912CA12CB12C06
:1026B000082E04C0880C991CAA1CBB1C0A94D2F7D3
:1026C000C4FE14C00FE010E020E030E0B901A80122
:1026D00004C0440F551F661F771F8A95D2F7CB01A0
:1026E000BA01609570958095909503C060E070E0A8
:1026F000CB01272D26952695237030E02230310519
:1027000069F02330310589F0682979298A299B29C4
:102710002130310571F00E94BD18DEC06829792989
:102720008A299B290E94D918D7C00E94BD18C501CB
:10273000B4010E94A118D0C0112319F0872D817017
:1027400001C08695882309F4C7C08C2D8295869593
:102750008770880F880F9C2D9F70892E912CA12C3B
:10276000B12C082E04C0880C991CAA1CBB1C0A940E
:10277000D2F7C4FE14C00FE010E020E030E0B90151
:10278000A80104C0440F551F661F771F8A95D2F712
:10279000CB01BA01609570958095909503C060E07B
:1027A00070E0CB01272D269526952370422F50E00F
:1027B0004230510569F04330510589F06829792983
:1027C0008A299B294130510571F00E94971984C0D4
:1027D000682979298A299B290E94B3197DC00E9402
:1027E0009719C501B4010E947B1976C08C2D90E029
:1027F000FC01E05EF109E531F10508F050C0E05957
:10280000FF4F0C9407240C2D0F70872D8F7111230F
:1028100031F00E941419802F0E9471125DC00E9435
:102820003519802F0E94781257C0112339F00111F9
:1028300053C0872D8F710E945A194EC0023008F084
:102840004BC0F7CF112339F0872D8F710E941419D7
:1028500043C01123C9F3872D8F710E9435193CC0E5
:10286000112329F0872D8F710E94FF1835C00E9417
:10287000F51832C0112351F0172D1F71812F0E94BE
:10288000141963E0812F0E94281A26C081E00E945B
:10289000311A023008F182E00E94311A1DC0112362
:1028A00031F0002389F28C2D0E945A1115C00023AB
:1028B00091F28C2D0E9422120FC0472D4F706C2D6B
:1028C000C7010E9469050E94191806C0472D4F7064
:1028D0006C2DC7010E944606DD20F9F00E94241AE3
:1028E00080FD1BC0F70112820E941E1A0E9414195B
:1028F000C7010E949C140E941E1A0F90DF91CF9175
:102900001F910F91FF90EF90DF90CF90BF90AF900D
:102910009F908F907F900C9435190F90DF91CF91FD
:102920001F910F91FF90EF90DF90CF90BF90AF90ED
:102930009F908F907F9008950F931F93CF93DF9375
:10294000EC01888199812B813C81232BB9F09F3F39
:1029500011F48F3F99F0CE010E949E05882371F0FB
:10296000688179818A810E941A1A8C010E94CF198C
:102970000E949618B801CE010E947F12DF91CF917C
:102980001F910F9108950E94F21A0E94021B0E944B
:10299000C71A0E941C1B0E9435200E94841F80E0E1
:1029A00090E00E94601080E090E00C9476100E940D
:1029B000E21A0C94C3140E940F1A292F22952F702B
:1029C00030E02C3031054CF42A3031056CF42250C3
:1029D000310922303105A8F407C02C30310569F0E7
:1029E0002F30310551F00DC0803F69F018F4803E62
:1029F00040F409C0843F29F406C093FB882780F97E
:102A0000089580E0089581E00895CF93DF9300D08A
:102A100000D01F92CDB7DEB70F900F900F900F90A0
:102A20000F90DF91CF910895CF93DF9300D000D026
:102A300000D0CDB7DEB726960FB6F894DEBF0FBE36
:102A4000CDBFDF91CF9108951F93CF93DF93C091B6
:102A5000850116E080918601C81799F0D0E01C9F8F
:102A6000F0011D9FF00D1124E957FE4F4081518167
:102A700062817381848195810E9414152196C770AB
:102A8000E9CFDF91CF911F9108954091B701509107
:102A9000B8016091B9017091BA018091BB01909128
:102AA000BC010C9414158091BC0182958F7009F0C3
:102AB00054C08091B901882309F44FC080918501E9
:102AC000A09186016091B7017091B8014091BA015F
:102AD0005091BB01B6E08A1709F43FC090E0411560
:102AE0005105C1F17F3F11F46F3FA1F1B89FF00193
:102AF000B99FF00D1124E957FE4F218172132AC0AE
:102B00002081621327C02281211124C023813481B6
:102B10002417350710F421503109241B350B283CAC
:102B20003105C0F42091BC012F7020612093BC01BD
:102B300026E0289FF001299FF00D1124E457FE4F55
:102B400080818F708061808387EB91E00E949C146C
:102B50000C94241501968770BECF0895CF92DF9212
:102B6000EF92FF920F931F93CF93DF93CDB7DEB712
:102B700062970FB6F894DEBF0FBECDBF8C0185E023
:102B8000F801DE011D9601900D928A95E1F7D801BA
:102B90004C9111965C91119712966C911297139625
:102BA000CD90DC9014973091B7017091B80180916D
:102BB000BA019091BB01009709F46BC17F3F19F4F2
:102BC0003F3F09F466C1E090B901EE2009F4C0C0AE
:102BD0002091BC01C816D90628F0F601E81BF90BB4
:102BE000CF0104C0809590958C0D9D1DFF24F3941A
:102BF000883C910578F0F12C207F09F0C6C07C2D2F
:102C0000D98AC88A89890E94051587EB91E00E94BC
:102C10009C14B1C0822F807F09F046C0751314C088
:102C2000341312C0611110C02F7020612093BC01B9
:102C30000E94451587EB91E00E949C148091BC0195
:102C4000D80115968C932EC0CD2819F15F3F11F451
:102C50004F3FF9F0F62E61111CC080918501209143
:102C6000860136E0821709F45AC090E0389FF001DF
:102C7000399FF00D1124E957FE4F7181571306C09B
:102C80007081471303C07281711103C00196877070
:102C9000E9CFF62E662309F418C18091BC0181604A
:102CA0008093BC01F12C11C1751308C0341306C008
:102CB000611104C08091BC01D801C3C04D875E87FB
:102CC0008D859E856A8B0E94DB146A898823E1F1D9
:102CD0006623D1F12091BC01822F82958F7090E004
:102CE000029774F08091B7019091B80198878F8313
:102CF0001986DB86CA862C87CE0107960E949C1413
:102D000086E0F801A7EBB1E001900D928A95E1F71A
:102D10000E9453150E944515FF24F394D6C04D8799
:102D20005E878D859E850E940F1A292F22952F7010
:102D300030E0223031050CF0BCC09F7009F0B6C005
:102D4000805E883008F4C1C0C8010E949C14E4CFA2
:102D5000C816D90608F453C0F601E81BF90BCF01D9
:102D6000883C910508F450C0F12C7C2DD98AC88A82
:102D700089890E940515E7EBF1E086E0DF011D92ED
:102D80008A95E9F70E944515A0C0751314C0341345
:102D900012C0611110C08091BC01F8018583C80187
:102DA0000E949C1486E0E7EBF1E0DF011D928A951A
:102DB000E9F7FE2C8AC04D875E878D859E856A8BDC
:102DC0000E94DB146A89882309F4BECF662309F4C4
:102DD000BBCF2091BC01822F82958F7090E002972B
:102DE0000CF48ECF8091B7019091B8019A838983BA
:102DF0001B82DD82CC822E83CE0101967FCF80950F
:102E000090958C0D9D1DACCFF62E662309F49CCFBA
:102E100075132EC034132CC02091BC0120FD1FC09F
:102E2000822F82958F70D9F0D80115962C93159723
:102E30008F3049F08F5F982F9295907F822F8F70FF
:102E4000892B15968C93C8010E949C1486E0F8018A
:102E5000A7EBB1E001900D928A95E1F793CF86E060
:102E6000F801A7EBB1E001900D928A95E1F72DC032
:102E70004D875E878D859E850E94DB14811140CF32
:102E80008091BC0181608093BC01C8010E949C14A8
:102E90001CC0662309F458CF4D875E878D859E85BB
:102EA0000E94DB14882309F44FCF2ACF811148CF29
:102EB0000CC0243031050CF047CF9F7009F440CF8F
:102EC000F8019581907F09F03BCF8F2D62960FB668
:102ED000F894DEBF0FBECDBFDF91CF911F910F9150
:102EE000FF90EF90DF90CF9008951F93CF93DF93E3
:102EF000CDB7DEB72C970FB6F894DEBF0FBECDBFAF
:102F00004F83588769877A878B879C87CE0107967E
:102F10000E94AE15882369F08F8198852A853B85AC
:102F2000232BF1F19F3F09F063C08F3F09F060C090
:102F300037C086E0FE013796DE01119601900D92B2
:102F40008A95E1F76F817885EA85FB85309741F1B5
:102F50007F3F11F46F3F21F12091860130E0C901DC
:102F60000196877099274091850150E08417950755
:102F700009F447C069837A83FD83EC8396E0929FCE
:102F8000D001939FB00D1124A957BE4FFE01319679
:102F900001900D929A95E1F7809386010E94241585
:102FA00016E080918501909186018917C1F1189FE3
:102FB000C001112489579E4F0E94AE15882379F1D4
:102FC000E09185011E9FF0011124E957FE4F4081D9
:102FD000518162817381848195810E941415809151
:102FE000850190E001968770992780938501D9CF5C
:102FF0004F81588569857A858B859C850E9414153B
:10300000CFCF0E94D7141092860110928501E7EB72
:10301000F1E086E0DF011D928A95E9F7C1CF2C9699
:103020000FB6F894DEBF0FBECDBFDF91CF911F91D9
:103030000895EF92FF920F931F93CF93DF938C012C
:10304000009709F46CC0F12CEE24E394E80121967A
:10305000F8018491843740F4843008F051C0813005
:1030600081F0823019F15BC0853709F444C0A8F1C2
:103070009CE7980F903708F052C08F770E94221279
:1030800041C00E5F1F4FFE01C49180E28C0F88305B
:1030900048F4C7708E2D01C0880FCA95EAF70E94C8
:1030A000F51A14C08C2F0E945A112DC00E5F1F4FAD
:1030B000FE01C49180E28C0F883058F4C7708E2DC9
:1030C00001C0880FCA95EAF70E94FB1A0E941C1BD8
:1030D0001AC08C2F0E94221216C00E5F1F4FFE01D5
:1030E000C491CC2381F08FE99FE00197F1F700C0F4
:1030F0000000C150F6CF0E5F1F4FFE01F49003C0D9
:103100000E945A118E018F2D882309F49FCFEFE979
:10311000FFE03197F1F700C000008150F5CFDF915B
:10312000CF911F910F91FF90EF90089508956093B4
:10313000C1017093C2018093C3019093C4010C94A8
:10314000C3140F931F930091C1011091C2012091EC
:10315000C3013091C401DC01CB01802B912BA22B48
:10316000B32B8093C1019093C201A093C301B0938C
:10317000C4011F910F910C94C3140F931F930091DE
:10318000C1011091C2012091C3013091C401DC0141
:10319000CB0180239123A223B3238093C101909379
:1031A000C201A093C301B093C4011F910F910C946D
:1031B000C3140F931F930091C1011091C20120917C
:1031C000C3013091C401DC01CB0180279127A227E4
:1031D000B3278093C1019093C201A093C301B09320
:1031E000C4011F910F910C94C3141092BD01109251
:1031F000BE011092BF011092C0010C94C31441E0B3
:1032000050E060E070E004C0440F551F661F771F58
:103210008A95D2F74093BD015093BE016093BF01E0
:103220007093C0010C94C31441E050E060E070E082
:1032300004C0440F551F661F771F8A95D2F78091EF
:10324000BD019091BE01A091BF01B091C001482B7A
:10325000592B6A2B7B2B4093BD015093BE01609389
:10326000BF017093C0010C94C31441E050E060E0D2
:1032700070E004C0440F551F661F771F8A95D2F770
:1032800040955095609570958091BD019091BE01DB
:10329000A091BF01B091C001482359236A237B2329
:1032A0004093BD015093BE016093BF017093C00174
:1032B0000C94C31441E050E060E070E004C0440F9F
:1032C000551F661F771F8A95D2F78091BD01909197
:1032D000BE01A091BF01B091C001482759276A27BC
:1032E0007B274093BD015093BE016093BF01709353
:1032F000C0010C94C3140F931F930091BD01109152
:10330000BE012091BF013091C001DC01CB01802BB7
:10331000912BA22BB32B8093BD019093BE01A09360
:10332000BF01B093C0011F910F910C94C3140F9370
:103330001F930091BD011091BE012091BF013091FA
:10334000C001DC01CB0180239123A223B32380930E
:10335000BD019093BE01A093BF01B093C0011F9126
:103360000F910C94C3140F931F930091BD01109102
:10337000BE012091BF013091C001DC01CB0180274B
:103380009127A227B3278093BD019093BE01A093FC
:10339000BF01B093C0011F910F910C94C314089505
:1033A000CF92DF92EF92FF920F931F93CF93DF9311
:1033B0008C01C090C101D090C201E090C301F09097
:1033C000C4018091BD019091BE01A091BF01B09157
:1033D000C001C82AD92AEA2AFB2ACFE1D0E0D701C6
:1033E000C6010C2E04C0B695A795979587950A94AB
:1033F000D2F780FF06C0B8018C2F0E949C0801976D
:1034000021F4219760F780E001C08C2FDF91CF91EC
:103410001F910F91FF90EF90DF90CF900895CF9381
:10342000DF93EC010E94D019BE010E949C08DF913D
:10343000CF910895CB010E940F1A08958091C50184
:1034400085958595859508958091C5018770089526
:1034500098E0899F90011124262B2093C5010C949C
:1034600014192091C501809582238093C501982F5E
:10347000977069F430E0482F552747FD5095241781
:10348000350729F08595859585950C94351908950E
:103490009091C501977081E009F480E008959091C2
:1034A0000C01992321F090910D01911109C02091F7
:1034B0000E0130910F01F90132969FEF40E01FC0DD
:1034C000982F9695969596959F3050F5E0910E0120
:1034D000F0910F01E90FF11D877021E030E0A901A3
:1034E00002C0440F551F8A95E2F7CA019181892BCA
:1034F000818308959F3F39F04F5F4E3041F05191E5
:103500005813F8CF0DC05111F7CF942FF5CF9F3F2F
:1035100039F0F901E90FF11D97FDFA9582830895BD
:10352000089590910C01992321F090910D01911132
:1035300009C020910E0130910F01F9013296205FF0
:103540003F4F1FC0982F9695969596959F30F0F413
:10355000E0910E01F0910F01E90FF11D877021E05C
:1035600030E0A90102C0440F551F8A95E2F7CA0155
:10357000809591818923818308953196E217F3071D
:1035800029F090819813F9CF1082F7CF089581E048
:1035900090E0E0910E01F0910F01E80FF91F108209
:1035A000019680319105A9F708959091D901892B51
:1035B0008093D901089580959091D90189238093B2
:1035C000D90108951092D90108959091D801892BBD
:1035D0008093D801089580959091D8018923809394
:1035E000D80108951092D80108959091D701892BA0
:1035F0008093D701089580959091D7018923809376
:10360000D70108951092D70108958093C6010895B7
:103610001092C601089580910E0190910F01FC0156
:1036200031969C01205F3F4F80E0919191118F5F17
:10363000E217F307D1F70895E0910E01F0910F0121
:103640008091D9018083E0910E01F0910F0190816A
:103650008091D801892B8083E0910E01F0910F01B8
:1036600090818091D701892B80838091C601882326
:1036700061F0E0910E01F0910F019081892B808320
:103680000E940B1B81111092C60180910E01909136
:103690000F010C944A1020E0009739F0AC01415022
:1036A0005109842395232F5FF7CF822F0895CF925E
:1036B000DF92EF92FF926C01EE24FF24C114D1043B
:1036C000E104F10421F0C701B60120E101C020E0CE
:1036D000C72ED82EE92EFF24C114D104E104F10431
:1036E00019F0285FC701B6016B017C0154E0F69424
:1036F000E794D794C7945A95D1F7C114D104E10443
:10370000F10419F02C5FC701B6016B017C0142E0A6
:10371000F694E794D794C7944A95D1F7C114D1048D
:10372000E104F10419F02E5FC701B601DC01CB0101
:10373000B695A79597958795892B8A2B8B2B09F0A2
:103740002F5F822FFF90EF90DF90CF9008958091B0
:10375000F101843021F11092DB0120E488E190E056
:103760000FB6F894A895809360000FBE2093600078
:1037700080E00E94370983B7817F846083BF83B76D
:10378000816083BF7894889583B78E7F83BF88E1FB
:103790000FB6F89480936000109260000FBE0895F9
:1037A000089508950E94D01B0E949F030E94D11B80
:1037B0000E94940491E0811101C090E0892F089546
:1037C0000E94D7140E943E100C94370982E084BDF9
:1037D00093E095BD9AEF97BD80936E0008952FB743
:1037E000F8948091DC019091DD01A091DE01B0910F
:1037F000DF012FBF0895CF92DF92EF92FF920F93D8
:103800001F932FB7F8944091DC015091DD01609136
:10381000DE017091DF012FBF6A017B01EE24FF24DE
:103820008C0120E030E0C016D106E206F30610F469
:10383000415051099A01281B390BC9011F910F9161
:10384000FF90EF90DF90CF9008951F920F920FB6E8
:103850000F9211248F939F93AF93BF938091DC01BC
:103860009091DD01A091DE01B091DF010196A11DD3
:10387000B11D8093DC019093DD01A093DE01B09334
:10388000DF01BF91AF919F918F910F900FBE0F906D
:103890001F9018950E943B0DF8942FEF87EA91E650
:1038A000215080409040E1F700C0000087E090EB9D
:1038B000DC018093FB019093FC01A093FD01B09388
:1038C000FE019CE088E10FB6F894A8958093600013
:1038D0000FBE90936000FFCFEF92FF920F931F9364
:1038E000CF93DF93D82FCDE08C2F0E948D0405E07D
:1038F00010E0E82EF12CC701002E02C095958795A7
:103900000A94E2F780FF09C0602F7C2F80E00E94BC
:103910004706D81302C081E006C00150110958F7CC
:10392000C15010F780E0DF91CF911F910F91FF9070
:10393000EF900895CF93C82F8CE20E946C1C8823CF
:1039400021F08C2FCF910C946C1C80E0CF910895C6
:10395000CF930E94EF1D811102C00E94D51DC5E6C4
:10396000C15049F00E949F038FE39CE90197F1F752
:1039700000C00000F5CF89E20E949A1C811113C19A
:103980008AE20E949A1C81110E94D51D85E00E9446
:103990009A1C81110E944A1C0E94FA1D8093DA0130
:1039A00087E00E949A1C8823A9F18BE10E949A1C4F
:1039B000882351F08091DA0181FB222720F991E0E0
:1039C000922790FB81F90EC08EE00E949A1C8823FA
:1039D00061F08091DA0182FB222720F991E09227A1
:1039E00090FB82F98093DA0115C080E10E949A1C55
:1039F0009091DA01882341F093FB222720F981E09E
:103A0000822780FB93F904C0892F809580FB90F971
:103A10009093DA018091DA010E94FE1D0E940C1E33
:103A20008093FA0180EE0E949A1C882341F08091D5
:103A3000FA01982F909590FB80F98093FA0189E321
:103A40000E949A1C882359F08091FA0181FB222759
:103A500020F991E0922790FB81F98093FA0182EEA0
:103A60000E949A1C882359F08091FA0182FB222738
:103A700020F991E0922790FB82F98093FA0186EE7B
:103A80000E949A1C882359F08091FA0183FB222717
:103A900020F991E0922790FB83F98093FA0183EE5D
:103AA0000E949A1C882359F08091FA0184FB2227F6
:103AB00020F991E0922790FB84F98093FA0185E345
:103AC0000E949A1C882359F08091FA0185FB2227D5
:103AD00020F991E0922790FB85F98093FA0181E328
:103AE0000E949A1C882359F08091FA0186FB2227B4
:103AF00020F991E0922790FB86F98093FA0181E109
:103B00000E949A1C882359F08091FA0187FB222792
:103B100020F991E0922790FB87F98093FA01809138
:103B2000FA010E94101E8091FA0187FB882780F914
:103B300080930D0187E20E949A1CC82F8EE10E949B
:103B40009A1C8111C2608FE10E949A1C8111C4608D
:103B500080E20E949A1C8111C86081E20E949A1C36
:103B60008111C06182E20E949A1C8111C06283E2CD
:103B70000E949A1C8111C06484E20E949A1C8823CE
:103B800011F0C06802C0CC2329F08C2F0E94071EC0
:103B90006C2F03C00E94031E682F70E080E090E04D
:103BA000CF910C949718CF9108956DEE7EEF80E041
:103BB00090E00E94412460E082E090E00E942F2487
:103BC00060E083E090E00E942F2460E084E090E0D9
:103BD0000E942F2460E085E090E00C942F2480E088
:103BE00090E00E94292421E08D3E9E4F09F020E0C4
:103BF000822F089582E090E00C942124682F82E0C7
:103C000090E00C942F2483E090E00C942124682F02
:103C100083E090E00C942F2484E090E00C94212425
:103C2000682F84E090E00C942F248091E20180FFC3
:103C30000BC06091130185E0689FB0011124759558
:103C40006795759567952BC081FF09C06091130139
:103C500085E0689FB00111247595679520C082FFAB
:103C600007C06091130185E0689FB001112417C05F
:103C70009091E3019923D1F060911201961788F792
:103C80002091130185E0289F90011124929FA001AB
:103C9000939F500D112470E0CA010E94F3236038F5
:103CA000710540F46115710539F002C065E070E0FE
:103CB000862F08958FE7089581E008958091E201AD
:103CC00080FF08C06091110170E07595679575954A
:103CD000679521C081FF06C06091110170E0759564
:103CE000679519C082FF04C06091110170E010C097
:103CF0009091E3019923C1F0609110019617A0F70C
:103D000080911101899FC001112470E00E94F3236A
:103D10006038710528F46115710521F0862F08952A
:103D20008FE7089581E0089561E070E0F4CF803F6F
:103D300021F40E94151E819504C0813F29F40E9440
:103D4000151E8093E6010895823F21F40E94151EFE
:103D5000819504C0833F29F40E94151E8093E501DC
:103D60000895893F19F40E945E1E05C08A3F31F410
:103D70000E945E1E81958093E70108958B3F21F498
:103D80000E945E1E819504C08C3F29F40E945E1E35
:103D90008093E8010895843F21F48091E4018160DB
:103DA00017C0853F21F48091E401826011C0863FF5
:103DB00021F48091E40184600BC0873F21F480915D
:103DC000E401886005C0883F31F48091E40180619E
:103DD0008093E40108958D3F21F48091E201816098
:103DE0000BC08E3F21F48091E201826005C08F3FBD
:103DF00029F48091E20184608093E2010895803F7C
:103E000039F48091E60187FF6CC01092E60169C029
:103E1000813F29F48091E6011816BCF362C09091AD
:103E2000E501823F29F497FF5CC01092E50159C07B
:103E3000833F19F41916CCF354C0893F41F48091A3
:103E4000E70118160CF04DC01092E7014AC08A3FF6
:103E500029F48091E70187FF44C0F6CF8B3F39F406
:103E60008091E80187FF3DC01092E8013AC08C3F85
:103E700029F48091E8011816BCF333C0843F21F483
:103E80008091E4018E7F17C0853F21F48091E40189
:103E90008D7F11C0863F21F48091E4018B7F0BC0A0
:103EA000873F21F48091E401877F05C0883F31F48A
:103EB0008091E4018F7E8093E40113C08D3F21F453
:103EC0008091E2018E7F0BC08E3F21F48091E20150
:103ED0008D7F05C08F3F29F48091E2018B7F809315
:103EE000E2018091E50181110EC08091E60181110E
:103EF0000AC08091E701811106C08091E80181111B
:103F000002C01092E301089584EE91E00E945510E2
:103F10000E94EF1B9093E1018093E00108951F93AD
:103F2000CF93DF938091E0019091E1010E94FB1B10
:103F3000AC019091E301992321F02091140130E02C
:103F400006C0209115018AE0289F90011124421794
:103F5000530708F486C08091E501C091E601D09135
:103F6000E7011091E801811107C0C11176C0D1119C
:103F700074C0111172C075C09F3F19F09F5F90937C
:103F8000E301181624F40E94151E8093E501809128
:103F9000E50187FF05C00E94151E81958093E5010C
:103FA0001C1624F40E94151E8093E6018091E60100
:103FB00087FF05C00E94151E81958093E6016091E0
:103FC000E501662339F1C091E601CC2319F1772789
:103FD00067FD7095872F972F0E94042323E333E317
:103FE00043E35FE30E9468230E94D1226093E501CE
:103FF0006C2F772767FD7095872F972F0E940423DA
:1040000023E333E343E35FE30E9468230E94D1226A
:104010006093E6011D1624F40E945E1E8093E70162
:104020008091E70187FF05C00E945E1E8195809305
:10403000E701111624F40E945E1E8093E80180912E
:10404000E80187FF05C00E945E1E81958093E8010C
:10405000DF91CF911F910C94841F9F3F09F08ECF69
:1040600096CFDF91CF911F910895E4EEF1E085E0C6
:10407000DF011D928A95E9F71092E3011092E201A7
:104080000895833081F128F4813059F08230D1F0E5
:104090000895853009F449C0B8F1863009F456C056
:1040A000089580911501262F30E0280F311D2F3FF4
:1040B000310524F4680F6093150108958FEF809304
:1040C0001501089580911401262F30E0280F311D2D
:1040D0002F3F310524F4680F6093140108958FEF8A
:1040E00080931401089580911301262F30E0280F4A
:1040F000311D2F3F310524F4680F6093130108959B
:104100008FEF80931301089580911201262F30E0E4
:10411000280F311D2F3F310524F4680F60931201E1
:1041200008958FEF80931201089580911101262F39
:1041300030E0280F311D2F3F310524F4680F6093C4
:10414000110108958FEF809311010895809110015E
:10415000262F30E0280F311D2F3F310524F4680F42
:104160006093100108958FEF8093100108958330BC
:1041700011F128F4813049F0823091F008958530B2
:1041800081F120F18630C1F1089580911501681701
:1041900020F4861B8093150108951092150108954F
:1041A00080911401681720F4861B809314010895F0
:1041B00010921401089580911301681720F4861B52
:1041C00080931301089510921301089580911201B4
:1041D000681720F4861B8093120108951092120133
:1041E000089580911101681720F4861B80931101B6
:1041F000089510921101089580911001681720F41C
:10420000861B8093100108951092100108950F935A
:104210001F938D3109F46BC008F03FC08E3009F454
:104220007FC0C0F4873009F469C068F4863009F0B3
:10423000B1C08091DA01817F8E7F8093DA0181E0C5
:104240008093EA01A8C0883009F4A2C08B3009F439
:104250009FC0A0C0863109F49BC078F4803109F476
:1042600072C0813109F096C00E94D71490910D015F
:1042700081E0892780930D018BC0893109F488C0C2
:104280008B3109F087C08091DA0181FB222720F968
:1042900091E0922790FB81F94CC0853309F470C0FE
:1042A00048F4873209F46CC008F459C0893209F423
:1042B00067C070C0833438F48A3308F04EC0883346
:1042C00009F466C067C0833409F45AC0883409F021
:1042D00061C00E94D7140FEF13ED20E3015010408E
:1042E0002040E1F700C000000E944A1C51C00E941B
:1042F0008B220E943E100E9437094AC09091DA0139
:10430000892F8095817080FB90F929F096609860E4
:104310009093DA0140C0997F977F9093DA0138C07B
:104320008091DA0182FB222720F991E0922790FB0D
:1043300082F98093DA01992359F18091DA01816041
:104340008093DA0125C08091DA0183FB222720F9CE
:1043500091E0922790FB83F9ECCF895301C08D51F6
:1043600041E050E060E070E08A019B0104C0000F72
:10437000111F221F331F8A95D2F7C901B80104C04B
:1043800061E070E080E090E00E9497180E94D714EE
:1043900081E001C080E01F910F91089580E00895B1
:1043A00080E00895CF93C82F8091EA01813079F0A1
:1043B00018F08230E9F187C0E0910E01F0910F0111
:1043C0008081813169F0823209F07FC009C0E091BB
:1043D0000E01F0910F018081813111F0823261F480
:1043E0008C2F0E94CE21811104C08C2F0E940721A6
:1043F0001DC081E090E01AC08C2F0E94D021811155
:1044000014C0C43179F048F4CB3079F0C03109F0F0
:1044100060C082E08093EA0108C0C93219F0C83355
:1044200021F057C01092EA0154C081E0817053C05E
:10443000C93289F118F5C43171F1A8F4C73009F017
:1044400046C08AE08093150194E19093140193E0B3
:10445000909313018093120188E08093110188E208
:104460008093100134C0CE51C63088F5EC2FF0E0B7
:10447000E65DFE4F80818093E90129C0CE34E9F0EA
:1044800020F4CB3421F56AE013C0C13579F0C23590
:10449000F1F461E00DC08091E901882319F01092D8
:1044A000E90115C081E08093EA0115C061E006C012
:1044B0008091E9010E9441200AC06AE08091E901EF
:1044C0000E94B72004C01092EA0180E004C081E09D
:1044D00002C080E0ABCFCF910895E1E8F0E08081A9
:1044E000886080838081816080838FB7F89493E0B7
:1044F0009093890090ED909388008FBF0895EFE628
:10450000F0E08081826080830895EFE6F0E08081B2
:104510008D7F80830895EFE6F0E0908182E0892727
:10452000808308951F920F920FB60F9211242F933C
:104530003F934F935F936F937F938F939F93AF932B
:10454000BF93EF93FF938091EB019091EC01019663
:104550009093EC018093EB01811103C082E00E94F3
:104560003709E091EC01E695E695F0E0E45AFA4F60
:10457000E4918091EB018E1303C080E00E94370923
:10458000FF91EF91BF91AF919F918F917F916F912B
:104590005F914F913F912F910F900FBE0F901F9001
:1045A000189504D06894B1118DC0089570D088F02A
:1045B0009F5790F0B92F9927B751A0F0D1F0660F0F
:1045C000771F881F991F1AF0BA95C9F712C0B1302A
:1045D00081F077D0B1E0089574C0672F782F8827D5
:1045E000B85F39F0B93FCCF3869577956795B39569
:1045F000D9F73EF490958095709561957F4F8F4FD8
:104600009F4F0895E89409C097FB3EF490958095DC
:10461000709561957F4F8F4F9F4F9923A9F0F92F88
:1046200096E9BB279395F695879577956795B79506
:10463000F111F8CFFAF4BB0F11F460FF1BC06F5FEC
:104640007F4F8F4F9F4F16C0882311F096E911C0FE
:10465000772321F09EE8872F762F05C0662371F01F
:1046600096E8862F70E060E02AF09A95660F771F33
:10467000881FDAF7880F9695879597F9089557FD63
:104680009058440F551F59F05F3F71F04795880FC0
:1046900097FB991F61F09F3F79F087950895121657
:1046A00013061406551FF2CF4695F1DF08C0161603
:1046B00017061806991FF1CF8695710561050894B4
:1046C0000895E894BB2766277727CB0197F90895CB
:1046D0000BD078C069D028F06ED018F0952309F07F
:1046E0005AC05FC01124EECFCADFA0F3959FD1F36B
:1046F000950F50E0551F629FF001729FBB27F00D90
:10470000B11D639FAA27F00DB11DAA1F649F6627E4
:10471000B00DA11D661F829F2227B00DA11D621F33
:10472000739FB00DA11D621F839FA00D611D221FED
:10473000749F3327A00D611D231F849F600D211DD1
:10474000822F762F6A2F11249F5750408AF0E1F074
:1047500088234AF0EE0FFF1FBB1F661F771F881FBD
:1047600091505040A9F79E3F510570F014C0AACF58
:104770005F3FECF3983EDCF3869577956795B795A8
:10478000F795E7959F5FC1F7FE2B880F911D9695D2
:10479000879597F9089597F99F6780E870E060E042
:1047A00008959FEF80EC089500240A9416161706CA
:1047B00018060906089500240A9412161306140612
:1047C00005060895092E0394000C11F4882352F075
:1047D000BB0F40F4BF2B11F460FF04C06F5F7F4F2D
:1047E0008F4F9F4F089597FB072E16F4009407D024
:1047F00077FD09D00E940D2407FC05D03EF490956A
:1048000081959F4F0895709561957F4F0895EE0FA4
:10481000FF1F0590F491E02D0994AA1BBB1B51E1E9
:1048200007C0AA1FBB1FA617B70710F0A61BB70B20
:10483000881F991F5A95A9F780959095BC01CD01C5
:104840000895F999FECF92BD81BDF89A992780B558
:104850000895A8E1B0E042E050E00C944924262FEE
:10486000F999FECF92BD81BDF89A019700B4021666
:1048700039F01FBA20BD0FB6F894FA9AF99A0FBE14
:1048800008950196272F0E9430240C942F24DC01D8
:10489000CB01FC01F999FECF06C0F2BDE1BDF89A4B
:1048A000319600B40D9241505040B8F70895F894F5
:0248B000FFCF38
:1048B20002203909C709A40970093C090101C7018D
:1048C20028080A03140A3F4D36391D05D0049A04FC
:1048D2006104F4030D0426043F04010203040506E7
:0448E20007080900BA
:00000001FF
